:100000000C9462000C948A000C948A000C948A0070
:100010000C948A000C948A000C948A000C9473143B
:100020000C948A000C948A000C948A000C94210C85
:100030000C948A000C948A000C948A000C948A0018
:100040000C94210E0C948A000C9462110C9494115F
:100050000C948A000C948A000C948A000C948A00F8
:100060000C94F40A0C948A000000000800020100BD
:100070000003040700000000000000000102040863
:100080001020408001020408102001020408102002
:10009000040404040404040402020202020203032E
:1000A0000303030300000000250028002B000000CC
:1000B0000000240027002A00020038021504EB0784
:1000C0009B0AC41111241FBECFEFD4E0DEBFCDBF09
:1000D00011E0A0E0B1E0EAEFFBE202C005900D9272
:1000E000AC35B107D9F723E0ACE5B1E001C01D9212
:1000F000A739B207E1F710E0C4ECD0E004C02297C2
:10010000FE010E94CF15CA3BD107C9F70E941715FF
:100110000C94FB150C9400002091640121110C94A7
:100120002B0520916701222339F0209165012111CF
:100130000C9417050C943E02089586E691E00E9407
:10014000DF0888E284B984E08AB926E040E05BE415
:1001500060E070E085EE92E00E9406110C948A0245
:100160000F931F9383B1837079F580915C01909117
:100170005D01A0915E01B0915F01892B8A2B8B2BD1
:1001800051F40E946B0E60935C0170935D0180934B
:100190005E0190935F010E946B0E00915C011091D3
:1001A0005D0120915E0130915F01601B710B820B3C
:1001B000930B693E73408105910570F08091650154
:1001C00091E089278093650110925C0110925D0196
:1001D00010925E0110925F011F910F910895DF92BE
:1001E000EF92FF920F931F93CF93DF9393B196FB00
:1001F000992790F9809167019817B1F183B186FB37
:10020000882780F98093670104E011E0C0E0D0E026
:10021000DD24D3947801F801219131918F01442795
:1002200037FD4095542F809167018D2590E0FC01AA
:10023000EE0FFF1FE80FF91FEC0FFD1FEE0FFF1F62
:10024000E65FFE4F6081718182E00E942F12F7010C
:1002500060817181882777FD8095982F0E949A0E82
:100260002196C330D105B1F6DF91CF911F910F9147
:10027000FF90EF90DF900895EF920F93E02E022F02
:10028000242F462F682F86E691E00E94FA080F91EE
:10029000EF900895CF92EF920F93CE2CE02E022F85
:1002A000242F462F682F86E691E00E9424090F91A3
:1002B000EF90CF900895CF93DF93EC010E940F0F42
:1002C0002F9781F4883C910554F1853823E09207FB
:1002D00064F5880F991F67E070E00E944315695329
:1002E000710925C0803921E0920754F484369105C4
:1002F000B4F063E070E00E9443156152710917C0C9
:10030000893522E0920774F0853823E092076CF477
:1003100063E070E00E9443156456710908C060E014
:1003200070E005C064E670E002C068EC70E0CB01EC
:10033000DF91CF910895CF92DF92EF92FF920F93CA
:100340008C3861F4E091E502F091E6020190F081D1
:10035000E02D65E585EE92E00995F4CF873861F5EB
:10036000E12C00E020E040E060E08FE90E944A01DB
:100370001E99FECF0E94770E6B017C011E9BFECF63
:100380000E94770E6C197D098E099F096C5772497E
:100390008109910924E130E040E050E00E947915A4
:1003A0002C593F4F4F4F5F4F2093600130936101B5
:1003B00040936201509363010F91FF90EF90DF90A3
:1003C000CF900895CF9389B1C3B1C770887FC82BF0
:1003D000C0958C2F0E949B01C0FD12C0C1FD12C0B0
:1003E000C2FD12C0C3FD12C0C4FD12C0C5FD12C0C3
:1003F0008C2F8074C6FD10C0C7FF0FC088E00DC0F1
:1004000081E00BC082E009C083E007C084E005C042
:1004100085E003C086E001C087E0CF91089583B1F5
:10042000881F8827881F809364010E94EF000E9424
:10043000B00080916401882319F00E942F0816C033
:1004400080916701882351F080916501882319F01C
:100450000E9419040BC00E94FE0208C088E285B900
:1004600064E670E080E090E00E949A0E0C94E20155
:100470006CE870E086E691E00C94C308FC01818191
:100480008A31F9F48681982F9278923811F410927B
:100490007501807A803A11F41092740181E095819F
:1004A000993C08F080E080937701882341F08091A7
:1004B0001601811106C081E08093760108951092A3
:1004C00076010895FC0140E09F01281B390B261797
:1004D00037071CF42191420FF7CF842F80950895A0
:1004E00081E080936E0180E180936F011092700132
:1004F0001092710164E070E08EE691E00E94620269
:100500008093720145E050E060E070E08EE691E09B
:100510000C94E31545E050E060E070E08EE691E079
:100520000E94D31564E070E08EE691E00E946202C2
:100530009091720189130C947002089564E070E048
:100540008EE691E00E9462028093720145E050E0E5
:1005500060E070E08EE691E00C94E315CF9389B1F2
:10056000C3B190911601911147C0C770887FC82B05
:10057000C09599F180916A018C132FC08091690117
:100580008F5F843118F4809369012BC01092690148
:100590008091680181111DC0C1FF10C080916E0162
:1005A00091E0892780936E011092760190937501F6
:1005B00084E1809373010E949E020BC08C2F857092
:1005C00041F081E08093750184E1809373010E9482
:1005D000700281E08093680104C01092680110925B
:1005E000690180917301882311F0815001C080E07E
:1005F00080937301C0936A01CF910895EF92FF92A7
:100600000F931F93CF93DF931F92CDB7DEB78EE08A
:1006100090E00E945B01182F8FE090E00E945B0148
:10062000282F80E190E029830E945B017C0181E119
:1006300090E00E945B01BC018091750129818111CC
:100640000AC080917401811108C080916E018823D5
:1006500031F005E005C001E803C008E801C001E091
:10066000A0916F01B0E084E6E81AF108EA9EA001CB
:10067000EB9E500DFA9E500D112486E0559547953E
:100680008A95E1F7E4E6F0E0E41BF50B8091700158
:10069000E80FF11D87FDFA95AB01445651094A9FB9
:1006A000B0014B9F700D5A9F700D112496E0759507
:1006B00067959A95E1F76C597F4F80917101680FAA
:1006C000711D87FD7A95123320F0173920F043E62B
:1006D00003C045E601C044E62093160180917701EE
:1006E000811102C020E004C0809176018823D1F3FB
:1006F00002608E2F0E943C0180917701882341F097
:1007000080917601882321F0809173018823F1F094
:1007100080916C0190916D01009721F0039721F079
:1007200085B103C088E201C080E085B980916C0189
:1007300090916D018530910511F0019602C080E025
:1007400090E090936D0180936C0108C080916E01E0
:10075000882311F088E001C080E285B90E94E2019F
:10076000882309F451C090916B0191114DC08130E3
:1007700029F4809375011092760148C0823049F4C3
:1007800090911601992309F43FC091E09093740170
:100790003BC08930C8F5843031F490916F019A31B3
:1007A00048F49F5F07C0833041F490916F01973008
:1007B00008F0915090936F0123C0873031F49091ED
:1007C00070019F304CF49F5F07C0863041F49091D8
:1007D0007001923F0CF091509093700111C08530E0
:1007E00031F4909171019F304CF49F5F07C08830C5
:1007F00039F490917101923F0CF0915090937101F6
:1008000089830E949E02898180936B010E94AE02BF
:1008100062E370E080E090E00F90DF91CF911F9154
:100820000F91FF90EF900C949A0E80E180936F01EE
:100830000895EF92FF920F931F93CF93DF9300D011
:10084000CDB7DEB78EE090E00E945B01282F8FE0ED
:1008500090E02A830E945B01082F80E190E00E94D3
:100860005B01182F81E190E00E945B0189830E9467
:10087000E201382F91E02A814981813009F090E02E
:1008800090937D01F0907C01911107C0011102C08D
:10089000FF2029F0E0917A0103C0E0E001C0E1E02F
:1008A000E0937A01F0917F01F13041F4F11032C010
:1008B000EE2381F1069544E664E631C0F530A1F4FB
:1008C00084E690E0811B910967E070E00E94431587
:1008D0006C59F11022C0EE2301F18BEA089F012D23
:1008E0001124069544E61BC01B3428F0612F1E37E7
:1008F00018F06DE701C06BE44B3420F04E3718F070
:100900004DE701C04BE4F11009C0EE2339F0069524
:10091000069505C044E664E601C044E600E08DEFBC
:10092000830F853038F5F1110AC08EEF830F809365
:100930007F0181E080937E0110927B0116C080913F
:100940007B01882391F0F13019F4363040F404C073
:10095000F23041F4353018F48EEF830F04C08091EB
:100960007E0101C081E080937E0181E080937D0162
:1009700010927A0190917F01992329F0311103C0DF
:1009800081E080937B01E0907E01E0917D019923DD
:1009900019F180E1E89E7001112480E8E89FF001E0
:1009A0001124EE2AE92A8BEA0E944A0180917C01F7
:1009B000811104C080917A0181110CC0809178016D
:1009C00090917901009721F0039771F480E011C0B4
:1009D00088E20FC015B80EC080917801909179011E
:1009E000009721F0039721F085B103C088E001C092
:1009F00080E285B9809178019091790185309105E7
:100A000011F0019602C080E090E09093790180930C
:100A1000780162E370E080E090E00F900F90DF914A
:100A2000CF911F910F91FF90EF900C949A0EFC01C3
:100A300021812A3B79F421E08581833D08F420E07F
:100A400020937C01211103C080917A0101C080E0D4
:100A500080937A010895CF93DF93EC010E946B0E8F
:100A600010929A011092990160938301709384010E
:100A7000809385019093860189818A3101F581E017
:100A80009D81993C08F080E08093DD01882361F02E
:100A90008091D80181110AC08091DC01811106C0CA
:100AA00081E08093DC0102C01092DC018A81809396
:100AB000DB018B818093DA018C818093D901DF91F6
:100AC000CF910895CF92DF92EF92FF920F931F93F1
:100AD000CF93DF9380EF8093A30104EA11E0CEE08F
:100AE000D0E0CE010E945B01F80181938F01219635
:100AF000C231D105B1F78091DB01FAE08F02C0016C
:100B0000112426E030E0B9010E944315E62F472F5B
:100B10008091DA015AE08502C0011124B9010E94D6
:100B200043152E2F342F2C398FEF380714F42CE96E
:100B30003FEFCB016C39EFEF7E0714F48CE99FEFA8
:100B40002536310514F024E630E02093AB018536DC
:100B5000910514F084E690E08093AC0180916001EF
:100B600090916101A0916201B09163010097A1058C
:100B7000B10511F0282F07C02091D9012F3F11F0A6
:100B80002F3108F02EE12093AA0139B123B127704B
:100B9000387F232B2093A80141E0209199013091C7
:100BA0009A01243131050CF040E04093A9012091D5
:100BB000DD01222329F021E03091DC01311101C057
:100BC00020E02093AD01181619061A061B0654F4EE
:100BD000E091E502F091E6020280F381E02D4BE026
:100BE00050E03FC089B190E023E0959587952A9524
:100BF000E1F78F708093AE0199B183B186958695A8
:100C00008E70991F9927991F890F8093AF0182E1F8
:100C10000E940F0F24E630E0DC010E94A715C12CD2
:100C200034E0D32EE12CF12CA70196010E94791516
:100C30002093B00183E10E940F0F24E630E0DC0135
:100C40000E94A715A70196010E9479152093B10172
:100C5000E091E502F091E6020280F381E02D4FE0A1
:100C600050E063EA71E085EE92E0DF91CF911F9151
:100C70000F91FF90EF90DF90CF9009940F931F9307
:100C8000CF93DF939091C6018091B301981771F0D3
:100C900085B190FF02C08F7D01C0806285B985B1AA
:100CA00091FF02C0877F01C0886085B9E091C701CC
:100CB0008091B401E817C1F08FEF8E0F8730A0F458
:100CC0002091C80184E6289F90011124442737FD14
:100CD0004095542FF0E0EE0FFF1FE95DFE4F60815D
:100CE000718182E00E942F12CEECD1E0EFE9F1E0B9
:100CF000ABE9B1E080E090E042E32991208331E06C
:100D0000211101C030E0832B332321F04C93253691
:100D100009F410823196119621E0C23DD20769F79D
:100D20009093980180939701892B39F081E090E0AE
:100D300090931801809317014BC08091C901909145
:100D4000B601891729F0893C08F088EC80931C01D2
:100D50008091CA019091B701891729F0893C08F068
:100D600088EC80931B018091CB019091B801891789
:100D700029F0893C08F088EC80931A018091CC011D
:100D80009091B901891799F08093D80181110BC016
:100D90008091DC01811107C08091DD01882319F069
:100DA00081E08093DC01109218011092170180916C
:100DB000CD019091BA01891759F0809319018138BA
:100DC00019F09091800198131092DC0180938001BA
:100DD0008091D2019091BF01891759F19AB181FF99
:100DE00002C0986001C0977F9AB99BB180FF02C092
:100DF000986001C0977F9BB99AB183FF02C0906150
:100E000001C09F7E9AB99BB182FF02C0906101C070
:100E10009F7E9BB99AB185FF02C0906201C09F7D01
:100E20009AB984FF03C08BB1806202C08BB18F7D01
:100E30008BB98091D3019091C001891759F19AB172
:100E400081FF02C0906401C09F7B9AB99BB180FF73
:100E500002C0906401C09F7B9BB99AB183FF02C01E
:100E6000906801C09F779AB99BB182FF02C09068D9
:100E700001C09F779BB994B185FF02C0986001C003
:100E8000977F94B984FF03C085B1886002C085B1A3
:100E9000877F85B9E091D4012091C1019E2F9227CF
:100EA0009F70E1F084B1E1FF02C0806101C08F7EDC
:100EB00084B985B1E0FF02C0806101C08F7E85B931
:100EC00084B1E3FF02C0806201C08F7D84B985B127
:100ED000E2FF02C0806201C08F7D85B98E2F82271C
:100EE000807739F42091D5018091C20128132DC05B
:100EF00042C0F0E043E0F695E7954A95E1F7EE70E1
:100F0000FF27E35EFE4F808191818093DE01909305
:100F1000DF0161E00E94B40F8091DE019091DF015A
:100F2000892B01F7CFE1D1E08E0160E070E088818C
:100F30000E942C0F229660E0F80180810E94B40F7D
:100F4000F1E0C732DF0781F7CDCFC091DE01D0914C
:100F5000DF011C161D067CF430E0AFEFB0E00E940C
:100F6000981524E630E040E050E00E947915B90180
:100F70008C2F0E942C0F6091D6018091C3016817BD
:100F800089F0662331F070E084E991E00E94770DEA
:100F900009C084E991E00E947D0D60E08091C30169
:100FA0000E94B40F6091D7018091C401681729F0A5
:100FB00070E084E991E00E94BC0D83E1E5ECF1E092
:100FC000A2EBB1E001900D928A95E1F7DF91CF910C
:100FD0001F910F91089584E991E00C94DD0CCF935B
:100FE000DF938091600190916101A0916201B091C5
:100FF0006301892B8A2B8B2B19F0CDE0D0E014C034
:10100000C3E1D0E011C085EE92E00E943C10803F29
:1010100021F410928201109281012091810130917E
:1010200082012C173D073CF085EE92E00E942310D0
:10103000892B49F711C0A9014F5F5F4F509382017F
:1010400040938101F901EB53FE4F80834C175D07FC
:1010500059F70E943E06E8CFDF91CF9108950F9394
:101060001F9380918C0181110DC00E946B0E6093C3
:1010700088017093890180938A0190938B0181E0AC
:1010800080938C010E946B0E009188011091890160
:1010900020918A0130918B01601B710B820B930BA5
:1010A000643171058105910508F469C00E946B0ED9
:1010B000609388017093890180938A0190938B01DA
:1010C0008091990190919A018436910514F40196CA
:1010D00002C084E690E090939A01809399010E9467
:1010E0006205EBE9F1E0AFE9B1E08081882319F016
:1010F0008150808301C01C923196119681E0EF39B6
:10110000F80799F78091990190919A014497BCF55D
:1011100000911901013811F41092D8012091870132
:1011200081E0282720938701809117019091180171
:101130002223A1F0009791F080919701909198015E
:10114000892B51F000EE2091A2014091A101609104
:10115000A00180919F0111C000EA07C0026073E006
:10116000880F991F7A95E1F7082B2091D8014091BB
:101170001A0160911B0180911C010E943C011F918A
:101180000F910C94EF071092F2017093E9016093B4
:10119000E80180EF8093EA0181EA8093EB0184E625
:1011A0008093EC018093ED018093EE011092EF01AA
:1011B00081E08093F0018EEC8093F101089566E761
:1011C00070E083EF91E00E948F0A6EE479E083EF94
:1011D00091E00E94960A61E779E083EF91E00E9436
:1011E000910A26E040E056E960E070E085EE92E08A
:1011F0000C940611EF920F938091F201811121C09E
:1012000081EA8093EB016093EC014093ED01209320
:10121000EE010093EF01E092F001EBEEF1E080E0EF
:101220009081903F09F49FEE9193890F91E0E13F07
:10123000F907B1F7803F09F48FEE8093F101109226
:10124000F2010F91EF900895CF92EF920F9380915A
:10125000F20181111FC06093EB014093EC012093D8
:10126000ED010093EE01E092EF01C092F001EBEE90
:10127000F1E09081903F09F49FEE9193890F91E006
:10128000E13FF907B1F7803F09F48FEE8093F10158
:101290001092F2010F91EF90CF9008958091F2019A
:1012A000882341F048E050E060EE71E083EF91E088
:1012B0000C94060A81E08093F20148E050E06AEE67
:1012C00071E083EF91E00E94060A88E0EAEEF1E027
:1012D000A0EEB1E001900D928A95E1F71092F20133
:1012E0000895CF92DF92EF92FF920F931F93CF93C7
:1012F000DF93CDB7DEB728970FB6F894DEBF0FBEE9
:10130000CDBF0897D1F48E010F5F1F4F7E0189E09A
:10131000E80EF11C680183EF91E00E94B409F80126
:1013200081938F01EE15FF05B1F7E091E801F0918F
:10133000E901309711F0C601099528960FB6F89487
:10134000DEBF0FBECDBFDF91CF911F910F91FF90F8
:10135000EF90DF90CF9008958091260290E0209149
:101360002702821B9109089520912702809126026D
:10137000281750F4E22FF0E0E85DFD4F808190E007
:101380002F5F2093270208958FEF9FEF0895E0913C
:10139000270280912602E81730F4F0E0E85DFD4F67
:1013A000808190E008958FEF9FEF08950895E09178
:1013B000FF01F09100023097E1F030912702209177
:1013C00026023217B0F040E0242F30E0261737070E
:1013D00054F4DC01A20FB31F5C91D901A85DBD4F8D
:1013E0005C934F5FF1CF1092270260932602CB01EE
:1013F00009940895E0910102F0910202309729F0DA
:10140000109205021092040209940895CF92DF927F
:10141000EF92FF920F931F93CF93DF937C01CB0149
:101420008A0120910302222389F0EB016B01C40E93
:10143000D51ECC15DD0569F06991D701ED91FC91C0
:101440000190F081E02DC7010995F3CF642F0E9430
:10145000C10AC801DF91CF911F910F91FF90EF90CA
:10146000DF90CF900895CF93DF931F92CDB7DEB773
:101470006983209103022223D1F0209104022032BB
:1014800040F021E030E0FC013383228380E090E0F3
:1014900015C080910502E82FF0E0EA5FFD4F9981C9
:1014A00090838F5F809305028093040205C061E002
:1014B000CE0101960E94C10A81E090E00F90DF9179
:1014C000CF910895FC011382128248EE53E060E050
:1014D00070E044835583668377838FE391E0918343
:1014E000808308951092270210922602109205021E
:1014F000109204020C949F0ACF93DF93EC01862F85
:101500000E94BD0A8AEF99E00E94DF0A87ED99E008
:101510000E94DA0ACE01DF91CF910C94720A0C94EA
:101520007C0A709300026093FF0108957093020299
:1015300060930102089583EF91E00C94620A109287
:10154000B50281E08093B3021092B20261E082E1C1
:101550000E94ED0F61E083E10E94ED0FE9EBF0E006
:1015600080818E7F808380818D7F808380E28093E5
:10157000B80085E48093BC000895880F8093BA007A
:101580000895613298F42091B502243089F4609373
:101590006A02FC018CE692E0DC012A2F281B261748
:1015A00018F421912D93F9CF80E0089581E00895FA
:1015B00082E008959093AF028093AE0208959093D5
:1015C000B1028093B002089585ED8093BC008091B4
:1015D000BC0084FDFCCF1092B502089585EC809389
:1015E000BC001092B50208951F920F920FB60F9291
:1015F00011242F933F934F935F936F937F938F9318
:101600009F93AF93BF93EF93FF938091B900887F2F
:10161000803609F49EC078F5883209F45DC090F4F4
:10162000803109F456C038F4882309F4F5C08830B5
:1016300009F44FC0F5C0883109F44EC0803209F476
:101640005FC0EEC0803409F46AC058F4803309F4F6
:1016500057C0883309F0E4C0809348020E94EE0A24
:10166000DFC0803509F44FC0883509F45DC0883487
:1016700009F0D6C0D3C0883909F4C4C0A8F48837AB
:1016800009F467C038F4883609F463C0803709F478
:1016900060C0C6C0883809F4B5C0803909F45FC09D
:1016A000803809F0BDC05BC0803B09F483C038F4CA
:1016B000803A09F466C0883A09F47CC0B1C0803C25
:1016C00009F4A4C0883C09F4A1C0883B09F487C090
:1016D000A7C08091B40210C090918D0280918C02BD
:1016E000981770F5E0918D0281E08E0F80938D0246
:1016F000F0E0E257FD4F80818093BB0085EC83C012
:10170000809348028BC0E0918D0281E08E0F809320
:101710008D028091BB00F0E0E257FD4F80839091F5
:101720008D0280918C026BC0E0918D0281E08E0F62
:1017300080938D028091BB00F0E0E257FD4F8083E3
:101740008091B30281116AC081E08093B20284EA81
:101750005EC083E08093B50210924902CFCF8091A2
:101760004902803208F04EC0E091490281E08E0FBC
:10177000809349028091BB00F0E0E65BFD4F8083DF
:10178000BDCF0E94EE0A80914902803230F4E09190
:101790004902F0E0E65BFD4F10826091490270E083
:1017A000E091AE02F091AF028AE492E009951092C6
:1017B000490236C084E08093B50210926B02109209
:1017C0006A02E091B002F091B102099580916A023B
:1017D000811105C081E080936A0210926C02E09151
:1017E0006B0281E08E0F80936B02F0E0E459FD4FB5
:1017F00080818093BB0090916B0280916A02981760
:1018000008F47CCF85E88093BC000AC085EC809307
:10181000BC001092B50204C0109248020E94E40A73
:10182000FF91EF91BF91AF919F918F917F916F91B8
:101830005F914F913F912F910F900FBE0F901F908E
:1018400018951F920F920FB60F9211242F933F936A
:101850004F935F936F937F938F939F93AF93BF93B8
:10186000EF93FF938091B70287FF05C01092850028
:10187000109284001AC02091B702332727FD3095BB
:101880008091B60290E0281739077CF48091B70266
:10189000992787FD9095FC01EE0FFF1FE80FF91FB8
:1018A000E854FD4F808186FD15C08091B7028F5F9F
:1018B0008093B7022091B702332727FD309580919E
:1018C000B60290E028173907BCF48091B7028C303B
:1018D0005CF112C08091B702992787FD9095FC01B9
:1018E000EE0FFF1FE80FF91FE854FD4F808160E005
:1018F0008F730E94ED0FD9CF809184009091850065
:10190000049680329E4418F480E29EE405C08091E3
:1019100084009091850004969093890080938800BC
:101920008FEF8093B70238C02091840030918500FA
:101930008091B702992787FD9095FC01EE0FFF1F5C
:10194000E80FF91FE854FD4F81819281820F931FA8
:1019500090938900809388008091B702992787FD32
:101960009095FC01EE0FFF1FE80FF91FE854FD4FA3
:10197000808186FF11C08091B702992787FD9095DD
:10198000FC01EE0FFF1FE80FF91FE854FD4F8081A7
:1019900061E08F730E94ED0FFF91EF91BF91AF91C6
:1019A0009F918F917F916F915F914F913F912F9177
:1019B0000F900FBE0F901F9018952091B6022C30FB
:1019C000A0F431E0320F3093B602FC012083822F65
:1019D00090E0FC01EE0FFF1FE80FF91FE854FD4FE8
:1019E0008CED95E09283818308952FEFFC01208395
:1019F0000895DF92EF92FF920F931F93CF93DF939F
:101A0000EC01D62E7A01890188818C3008F066C0FD
:101A100061E08D2D0E94B40F8881A82FB0E0FD01F8
:101A2000EE0FFF1FEA0FFB1FE854FD4F2D2D2F7304
:101A30009081907C922B908360E272E06E197F0916
:101A400077FF02C06D5F7F4F7595679575956795B8
:101A5000698340E659E0401B510B57FF02C04D5FC0
:101A60005F4F55954795559547954A836CE00E9481
:101A700037159CE0899FB001112420E030E0A901D6
:101A8000460F571FFA01EE0FFF1FE40FF51FE85432
:101A9000FD4F908196FD16C02F5F3F4F2C303105D2
:101AA00071F781110FC01092800082E08093810055
:101AB0001092850010928400B19A80916F0082602C
:101AC00080936F00888190E0FC01EE0FFF1FE80F0C
:101AD000F91FE854FD4F8081806480838881DF9105
:101AE000CF911F910F91FF90EF90DF90089520E626
:101AF00039E040E252E00C94F90CFC01808190E066
:101B0000FC01EE0FFF1FE80FF91FE854FD4F808125
:101B10008F7B80830895FC0180818C3060F59181FA
:101B200028E830E0291B310997FD3395220F331F38
:101B3000220F331F621773077CF0928128E532E091
:101B4000291B310997FD3395220F331F220F331FB5
:101B5000621773070CF49B014FB7F89490E0225082
:101B60003109FC01EE0FFF1FE80FF91FE854FD4F8C
:101B7000328321834FBF08954F925F926F927F927D
:101B8000AF92BF92CF92DF92EF92FF920F931F938B
:101B9000CF93DF93EC01603282E078070CF040C015
:101BA00077FD06C0653B71052CF064EB70E002C068
:101BB00060E070E0898128E830E0281B310987FD6A
:101BC0003395220F331F220F331F5901CC24B7FC4A
:101BD000C094DC2C882777FD8095982F2A8148E5D2
:101BE00052E0421B510927FD5395440F551F440FE6
:101BF000551F2A01662457FC6094762C7F926F92C1
:101C00005F924F9214EBE12EF12C00E010E020E007
:101C100030E0A9010E94CF140F900F900F900F9009
:101C2000CE01DF91CF911F910F91FF90EF90DF9048
:101C3000CF90BF90AF907F906F905F904F900C943B
:101C40008B0D1F920F920FB60F9211242F933F937B
:101C50008F939F93AF93BF938091DD029091DE02AB
:101C6000A091DF02B091E0023091DC0226E0230F68
:101C70002D3720F40296A11DB11D05C029E8230FC0
:101C80000396A11DB11D2093DC028093DD02909389
:101C9000DE02A093DF02B093E0028091E102909116
:101CA000E202A091E302B091E4020196A11DB11DF0
:101CB0008093E1029093E202A093E302B093E402E6
:101CC000BF91AF919F918F913F912F910F900FBE38
:101CD0000F901F9018952FB7F8946091DD027091C6
:101CE000DE028091DF029091E0022FBF08953FB79E
:101CF000F8948091E1029091E202A091E302B09108
:101D0000E40226B5A89B05C02F3F19F00196A11D3E
:101D1000B11D3FBF6627782F892F9A2F620F711D43
:101D2000811D911D43E0660F771F881F991F4A95FB
:101D3000D1F708958F929F92AF92BF92CF92DF9288
:101D4000EF92FF926B017C010E94770E4B015C01C8
:101D5000C114D104E104F104F1F00E9426150E949F
:101D6000770E681979098A099B09683E73408105D5
:101D7000910570F321E0C21AD108E108F10888EE5C
:101D8000880E83E0981EA11CB11CC114D104E1048B
:101D9000F10429F7DDCFFF90EF90DF90CF90BF9057
:101DA000AF909F908F900895789484B5826084BDA1
:101DB00084B5816084BD85B5826085BD85B581604F
:101DC00085BDEEE6F0E0808181608083E1E8F0E0AF
:101DD0001082808182608083808181608083E0E8DE
:101DE000F0E0808181608083E1EBF0E080818460BD
:101DF0008083E0EBF0E0808181608083EAE7F0E0BF
:101E000080818460808380818260808380818E7FF6
:101E100080838081806880831092C10008958E3015
:101E200008F08E5087702091390190E4299F90012D
:101E30001124822B80937C0080917A0080648093AF
:101E40007A0080917A0086FDFCCF80917800209105
:101E5000790090E0922B08951F93CF93DF93182F72
:101E6000EB0161E00E94B40F209711F460E004C020
:101E7000CF3FD10539F461E0812FDF91CF911F91E0
:101E80000C94ED0FE12FF0E0E859FF4FE491E330BF
:101E9000F9F048F4E130B9F0E230A1F584B58062A0
:101EA00084BDC8BD34C0E730E9F0E83019F1E43052
:101EB00049F580918000806280938000D0938B00F0
:101EC000C0938A0024C084B5806884BDC7BD1FC08C
:101ED00080918000806880938000D0938900C093B7
:101EE000880015C08091B00080688093B000C093D6
:101EF000B3000DC08091B00080628093B000C093A9
:101F0000B40005C0C038D1050CF0B5CFAFCFDF911C
:101F1000CF911F910895833081F028F4813099F09A
:101F20008230A1F008958730A9F08830B9F084306C
:101F3000D1F4809180008F7D03C0809180008F77E5
:101F400080938000089584B58F7702C084B58F7D1B
:101F500084BD08958091B0008F7703C08091B00058
:101F60008F7D8093B0000895CF93DF9390E0FC01C4
:101F7000E458FF4F2491FC01E057FF4F84918823E0
:101F800049F190E0880F991FFC01E255FF4FA591A0
:101F9000B4918C559F4FFC01C591D4919FB76111AD
:101FA00008C0F8948C91209582238C938881822399
:101FB0000AC0623051F4F8948C91322F309583230B
:101FC0008C938881822B888304C0F8948C91822B17
:101FD0008C939FBFDF91CF9108950F931F93CF9361
:101FE000DF931F92CDB7DEB7282F30E0F901E85913
:101FF000FF4F8491F901E458FF4F1491F901E05724
:10200000FF4F04910023C9F0882321F069830E94C7
:102010008B0F6981E02FF0E0EE0FFF1FEC55FF4FB3
:10202000A591B4919FB7F8948C91611103C010955C
:10203000812301C0812B8C939FBF0F90DF91CF91A3
:102040001F910F910895FC01818D228D90E0805C9D
:102050009F4F821B91098F7399270895FC01918DE1
:10206000828D981731F0828DE80FF11D858D90E0FB
:1020700008958FEF9FEF0895FC01918D828D981741
:1020800061F0828DDF01A80FB11D5D968C91928D5C
:102090009F5F9F73928F90E008958FEF9FEF089559
:1020A0008AEB91E1892B49F080E090E0892B29F0BF
:1020B0000E94BA1181110C9400000895FC01848DD6
:1020C000DF01A80FB11DA35ABF4F2C91848D90E062
:1020D00001968F739927848FA689B7892C93A0893D
:1020E000B1898C9180648C93938D848D981306C0F4
:1020F0000288F389E02D80818F7D80830895CF93BE
:10210000DF93EC01888D8823C9F0EA89FB898081FF
:1021100085FD05C0A889B9898C9186FD0FC00FB6D1
:1021200007FCF5CF808185FFF2CFA889B9898C9112
:1021300085FFEDCFCE010E945E10E7CFDF91CF91FA
:102140000895CF92DF92FF920F931F93CF93DF9367
:102150001F92CDB7DEB76C0181E0D60158968C9303
:1021600058975B969C915B975C968C915C979813C3
:1021700007C05096ED91FC915197808185FD2EC04E
:10218000F601038D10E00F5F1F4F0F731127F02E24
:10219000F601848DF81211C00FB607FCF9CFD601F5
:1021A0005096ED91FC915197808185FFF1CFC6014A
:1021B00069830E945E106981EBCF838DE80FF11D6A
:1021C000E35AFF4F6083D6015B960C935B97529660
:1021D000ED91FC915397808180620CC0D601569698
:1021E000ED91FC91579760835096ED91FC9151973A
:1021F00080818064808381E090E00F90DF91CF91B7
:102200001F910F91FF90DF90CF900895BF92CF92D2
:10221000DF92EF92FF92CF93DF93EC016A017B0193
:10222000B22E60E874E88EE190E0A70196010E946A
:102230005715215031094109510956954795379550
:102240002795E889F98982E08083211580E13807A4
:1022500098F0E889F989108260E472E48FE090E0F8
:10226000A70196010E9457152150310941095109D2
:102270005695479537952795EC85FD853083EE85F6
:10228000FF852083188EEC89FD89B082EA89FB895D
:10229000808180618083EA89FB8980818860808376
:1022A000EA89FB89808180688083EA89FB89808153
:1022B0008F7D8083DF91CF91FF90EF90DF90CF9063
:1022C000BF9008951F920F920FB60F9211242F9373
:1022D0008F939F93EF93FF93E091F502F091F602B5
:1022E0008081E091FB02F091FC0282FD12C090819E
:1022F0008091FE028F5F8F732091FF02821751F051
:10230000E091FE02F0E0EB51FD4F958F8093FE02CD
:1023100001C08081FF91EF919F918F912F910F903C
:102320000FBE0F901F9018951F920F920FB60F922D
:1023300011242F933F934F935F936F937F938F93CA
:102340009F93AF93BF93EF93FF9385EE92E00E942C
:102350005E10FF91EF91BF91AF919F918F917F910F
:102360006F915F914F913F912F910F900FBE0F9002
:102370001F90189585EE92E00E94231021E0892B92
:1023800009F420E0822F08951092E8021092E702EB
:1023900088EE93E0A0E0B0E08093E9029093EA0237
:1023A000A093EB02B093EC028FE491E09093E602ED
:1023B0008093E50285EC90E09093F2028093F10225
:1023C00084EC90E09093F4028093F30280EC90E030
:1023D0009093F6028093F50281EC90E09093F802DE
:1023E0008093F70282EC90E09093FA028093F902D6
:1023F00086EC90E09093FC028093FB021092FE0228
:102400001092FF0210920003109201030895CF92E0
:10241000DF92EF92FF920F931F93CF93DF937C0194
:102420006A01EB0100E010E00C151D0571F06991E7
:10243000D701ED91FC910190F081E02DC701099544
:10244000892B19F00F5F1F4FEFCFC801DF91CF919C
:102450001F910F91FF90EF90DF90CF9008953F92E2
:102460004F925F926F927F928F929F92AF92BF92A4
:10247000CF92DF92EF92FF920F931F93CF93DF9350
:1024800000D000D0CDB7DEB78B0129013A01909181
:102490003A01981721F09F3F09F0DAC104C0E8EB38
:1024A000F0E0349081C080933A01E8EBF0E0E491F1
:1024B000EF3F09F4CDC1E13031F1E23009F44BC016
:1024C000E11171C014BC15BC94B5926094BD95B572
:1024D000916095BD282F30E0F901E057FF4FE4915E
:1024E000F0E0EE0FFF1FEC55FF4F459154915093D4
:1024F000920340939103F901E458FF4F24912093F4
:102500009003312C53C01092800010928100909162
:1025100081009860909381009091810091609093E8
:102520008100282F30E0F901E057FF4FE491F0E0FF
:10253000EE0FFF1FEC55FF4F4591549150938B03C5
:1025400040938A03F901E458FF4F249120938903B3
:10255000332433942BC01092B0001092B1009091AC
:10256000B00092609093B0009091B1009160909310
:10257000B100282F30E0F901E057FF4FE491F0E07F
:10258000EE0FFF1FEC55FF4F45915491509384037C
:1025900040938303F901E458FF4F24912093820371
:1025A00052E0352E03C03E2E37FC52C161E00E943E
:1025B000B40F4801A12CB12C832D8D7F09F0C7C029
:1025C00060E079E08DE390E0A50194010E94791527
:1025D00029833A834B835C8369017A0181E0C81ABD
:1025E000D108E108F1089FEFC916D104E104F10414
:1025F00009F008F49AC060E271EA87E090E0A50172
:1026000094010E94791569017A01E1E0CE1AD1089E
:10261000E108F108F2E03F1219C08FEFC816D104AB
:10262000E104F10409F008F48AC068E478EE81E07E
:1026300090E0A50194010E94791569017A0191E069
:10264000C91AD108E108F10883E001C082E0EFEF88
:10265000CE16D104E104F10409F008F467C064E285
:1026600074EF80E090E0A50194010E947915690162
:102670007A01F1E0CF1AD108E108F1083320E1F046
:1026800082E038121BC09FEFC916D104E104F104A7
:1026900009F008F4DBC062E17AE780E090E0A50190
:1026A00094010E94791569017A01E1E0CE1AD108FE
:1026B000E108F10885E003C083E001C084E0FFEF9A
:1026C000CF16D104E104F10489F180F169E07DE3E2
:1026D00080E090E0A50194010E94791569017A01DA
:1026E00081E0C81AD108E108F108311002C084E085
:1026F00001C086E09FEFC916D104E104F104B1F0F6
:10270000A8F0C980DA80EB80FC809AE0F594E79429
:10271000D794C7949A95D1F7E1E0CE1AD108E10891
:10272000F108332031F087E00BC081E0332011F055
:1027300007C085E095B5987F982B95BD38C082E09D
:102740009091B100987F982B9093B10030C060E0D9
:1027500079E08DE390E0A50194010E94791569016B
:102760007A01F1E0CF1AD108E108F108C114D104CF
:1027700081E0E806F10488F064E274EF80E090E024
:10278000A50194010E94791569017A0191E0C91AA5
:10279000D108E108F10893E001C091E0E1E03E12C8
:1027A00006C080918100887F892B8093810041142D
:1027B00051046104710471F0D801AA0FBB1FA30179
:1027C00092010E94AE1528EE33E040E050E00E94F6
:1027D000571503C02FEF3FEFA901F1E03F16A1F01D
:1027E00082E0381619F1311033C0C7BC209393032F
:1027F00030939403409395035093960380916E0019
:10280000826080936E0024C0D0928900C0928800BC
:1028100020938C0330938D0340938E0350938F034A
:1028200080916F00826080936F0012C0C092B300ED
:102830002093850330938603409387035093880346
:102840008091700082608093700002C084E078CF35
:102850000F900F900F900F90DF91CF911F910F91DC
:10286000FF90EF90DF90CF90BF90AF909F908F90B0
:102870007F906F905F904F903F900895813039F036
:1028800018F0823051F0089510926E0008958091F2
:102890006F008D7F80936F000895809170008D7F11
:1028A0008093700081E08093B0008091B100887FB8
:1028B00084608093B1001092B3000895CF93C82F25
:1028C00080913A018C1307C0E8EBF0E084919FEF10
:1028D00090933A0101C08FEF0E943E1460E08C2F6C
:1028E000CF910C94ED0F1F920F920FB60F921124FF
:1028F0002F933F934F935F936F937F938F939F9308
:10290000AF93BF93EF93FF938091850390918603DC
:10291000A0918703B0918803892B8A2B8B2B51F1CF
:1029200090918203E0918303F09184038081892751
:1029300080838091850390918603A0918703B09155
:102940008803181619061A061B06C4F4809185031D
:1029500090918603A0918703B09188030197A10904
:10296000B1098093850390938603A0938703B09366
:10297000880304C080913A010E945E14FF91EF9198
:10298000BF91AF919F918F917F916F915F914F9187
:102990003F912F910F900FBE0F901F9018954F925F
:1029A0005F926F927F92AF92BF92CF92DF92EF923F
:1029B000FF920F931F93CF93DF93CDB7DEB729011B
:1029C0003A01621B730B840B950B29893A894B8959
:1029D0005C892A193B094C095D09298B3A8B4B8B81
:1029E0005C8B9B01AC0169897A898B899C890E94E7
:1029F0002715E418F50806091709A80197010E9490
:102A000079152A0D3B1D4C1D5D1DCA01B901DF91D1
:102A1000CF911F910F91FF90EF90DF90CF90BF90DB
:102A2000AF907F906F905F904F90089508950E94AF
:102A3000D40E0E9416150E949D00C0E5D0E10E94B0
:102A40000F022097E1F30E945010F9CF0895DB01A7
:102A50008F939F930E94AE15BF91AF91A29F800D5F
:102A6000911DA39F900DB29F900D11240895991B65
:102A700079E004C0991F961708F0961B881F7A9575
:102A8000C9F78095089597FB072E16F4009407D098
:102A900077FD09D00E94B91507FC05D03EF490954A
:102AA00081959F4F0895709561957F4F0895A1E29C
:102AB0001A2EAA1BBB1BFD010DC0AA1FBB1FEE1FB8
:102AC000FF1FA217B307E407F50720F0A21BB30B03
:102AD000E40BF50B661F771F881F991F1A9469F77F
:102AE00060957095809590959B01AC01BD01CF01DB
:102AF0000895052E97FB1EF400940E94901557FD33
:102B000007D00E94571507FC03D04EF40C94901583
:102B100050954095309521953F4F4F4F5F4F089509
:102B200090958095709561957F4F8F4F9F4F089539
:102B3000A29FB001B39FC001A39F700D811D1124FE
:102B4000911DB29F700D811D1124911D08950E9449
:102B50009815B7FF0895821B930B08950E9498154E
:102B6000A59F900DB49F900DA49F800D911D1124E1
:102B70000895AA1BBB1B51E107C0AA1FBB1FA617C4
:102B8000B70710F0A61BB70B881F991F5A95A9F716
:102B900080959095BC01CD010895EE0FFF1F059023
:102BA000F491E02D0994DC01CB01FC01F999FECFF1
:102BB00006C0F2BDE1BDF89A319600B40D924150C5
:102BC0005040B8F70895DC01CB0103C02D910E945D
:102BD000EE1541505040D0F70895262FF999FECFB9
:102BE0001FBA92BD81BD20BD0FB6F894FA9AF99A2A
:0A2BF0000FBE01960895F894FFCF80
:102BFA0001000000640064002C018801B801EE01A4
:102C0A00EE01B80188010101000164646400000357
:102C1A0000050006000B000000060126014A015DBE
:102C2A00018801B801EE010B0201FF000000003328
:102C3A000A060AAC09B409C709D60900000000A1AE
:0C2C4A0010071223103C102E107F100009
:00000001FF
